:100000004B220D30840052280B1D09009000030E76
:100010008F008312851D0E2891011328110F910066
:100020004220FF309C00051E172892011C28120F49
:1000300092004220FF309C00061C202893012428B7
:10004000061C130F930042201A081B0403192D28C5
:100050009B0F2D289A0F2D289D161708031D970317
:10006000180A031936281808031D98031C080319D9
:100070003C289C0B3C281D170F0E8300900E100E81
:100080000B110900FB309A00B4309B000800820776
:10009000583400344C340034203400344D34483467
:1000A0007A34003443308C008001840A8C0B54284D
:1000B0000130C10083161C308500033086000430F7
:1000C000810083128101A0308B00FE308600132155
:1000D000742242209D128F30EC200230F2208920C1
:1000E0009D1A69281D1780228E30EC2000301E1FBB
:1000F0007A280430F220233036225322253044223D
:100100002F2227304422222223303D22D3209B203D
:1001100070288A30EC200630F2200800442294280F
:1001200036225322B001B1012F225330B000983053
:10013000B100222208009D102E09C039031DA728F6
:100140009D14AE09AF090130AF070318AE0A2208AB
:10015000AD000310AE0D0310AF0D0318AE0A03106F
:10016000EB2193218030EC203830840009308C0062
:100170000008E220840A8C0BB8287930EC200008B3
:10018000E220080036228030AE0653228130B000D3
:100190009030B10022227E30B0007030B1002F22AA
:1001A0008030AE0608004D212330362220303D221B
:1001B000293044220B222921203036220800E12058
:1001C000E1202030A000A1008615FB280130EC20A2
:1001D00018304C2208008130A000A1008611FB20BD
:1001E000861508009F004720FF3903190800E22008
:1001F0001F08013EF228831601308600831206157F
:10020000F030A00506080E392004860006110615F8
:10021000A10EF030A10506080E3921048600061152
:100220004B308F21080086012421242124212830ED
:10023000860006114B222830EC200830EC20E62006
:100240000630EC200C30EC284B22383086000611AA
:1002500008001D129D156D224E30B0002030B100F7
:100260002F225230B0000830B10022222B3044221D
:10027000192203194A292B303D227421C2306621EC
:100280002E0866212F0866218E30662100306621F7
:1002900079211E131D1A9D1108001E1F51291808CF
:1002A00063217421C330662108308C008E218514AF
:1002B0008E21050C9E0D85108C0B56298A218021DC
:1002C00079211E1B63216E30980008009F000830C2
:1002D0008C009F0D03188A21031C852180218C0B23
:1002E00069298A218021080085148A218E2185218F
:1002F000822985218E2185148E218A218E21080054
:100300008E2185148E218510080005108316051096
:100310008312080083160514831208000F308D0025
:100320008D0B90290800031018308C00B901BB0117
:10033000BE01C001B60DB50DB40DC00DBE0DBB0D97
:10034000B90D8C0BC629400EBF003E0EBC003B0E03
:10035000BA00390EB8001D103830DB213930DB21EE
:100360003A30DB213B30DB213C30DB211D143E30B9
:10037000DB21A530BD003F30DB214030DB219D1C5F
:100380000800370884002D30800008004030CF215D
:100390003E30CF213B30CF213930CF219A29840004
:1003A000033000079F009F198000303000079F0036
:1003B0009F1B8000080084000F3000050319E4290A
:1003C000303E80001D1408001D18E02920308000F8
:1003D0000408B7000800B6012E08B4002F08B500C5
:1003E00008308C00AD0C0318FA298C0BF229B401EB
:1003F000B50108000310052AAD0C031C052A2F08BF
:10040000B5072E0803182E0FB407B40CB50CB60CA4
:100410008C0BFC2908003108AF0730080318300F97
:10042000AE0708003108AF023008031C300FAE02DF
:10043000080031082F029F003008031C300A2E02EA
:100440001F0408003008B2003108B3000130B107C2
:100450000318B00A1922031C08003230332A19226B
:1004600003180800303036221D16080084000008EA
:10047000AE00840A0008AF00080084002E08800047
:10048000840A2F088000080084000008B000840A55
:100490000008B100080076308D008E018E0B4E2AC8
:1004A0008D0B4E2A0800B001A5221D19C322410858
:1004B000C200C20B5C2A602AC20B5F2A622A642A2D
:1004C0000130662A5030662A0830662AB100AF2211
:1004D0001D190B22B9221D1912222E09C039031D24
:1004E0000800AE01AF010800890122308400093004
:1004F0008C0093228000890A840A8C0B792A0800D8
:100500001D1F08001D1389012230840009308C0052
:100510009322000203198E2A00089822890A840A6D
:100520008C0B882A08008316081483120808080018
:10053000880083160812081555308900AA308900F2
:100540008814081EA12A8312080016081302031833
:10055000AB2A1D15AC2A1D111308960008001408BB
:1005600011020318B52A1D15B62A1D111108940091
:100570000800150812020318BF2A1D15C02A1D11F4
:10058000120895000800C10B08000330C1000800E4
:02400E00FA3F77
:10420000FA00510040004E0020005200080000005B
:024210000000AC
:00000001FF
